:100000000C943E001895000018950000189500000B
:10001000189500001895000018950000189500002C
:10002000189500001895000018950000189500001C
:10003000189500001895000018950000189500000C
:1000400018950000189500001895000018950000FC
:1000500018950000189500001895000018950000EC
:1000600018950000189500001895000018950000DC
:100070001895000018950000189500008FEF8DBFAF
:10008000C8EDE0EC4E2E80E18EBFD0E1F0E15F2EB6
:10009000A89584B7082E877F84BF88E1992780932D
:1000A000600090936000EEEFFFE0A0E0B1E08827F1
:1000B0008D933197E9F787E08093C40080E08093C7
:1000C000C50088E18093C100662487E880937A00A8
:1000D00080E080937C003B9A219A3C9A3A9A399A24
:1000E000549A3D9A389A539A209A559A3F9A239A4D
:1000F000099A3E9A0D9A229A579A569A02E010E06F
:1001000020E030E0AEE1B1E00D931D932D933C93E0
:1001100002E518EB2EE135E0A8E0B1E00D931D9368
:100120002D933C9381E08093000184E08093010152
:1001300083E08093140180E08093020185E0809346
:1001400003012A9AE1E0F0E00E94D513459AE1E02C
:10015000F0E00E94D513409844985C985B9A2998E7
:10016000479A2B9A1198449A81E090E00E94E413F8
:1001700044983A9A3B9A4398A0E0B1E0119698E0EF
:100180008E91983018F4392F992702C038E0985092
:10019000881F429808F4429A00000000439AEF93A7
:1001A000FF93EFE0F0E00E94DB13FF91EF914398A3
:1001B000EF93FF93EFE0F0E00E94DB13FF91EF91EC
:1001C0003A9531F79923E1F683ED809311013A9A3C
:1001D0003B9A4398A1E1B1E0119698E08E91983056
:1001E00018F4392F992702C038E09850881F429898
:1001F00008F4429A00000000439AEF93FF93E6E46C
:10020000F0E00E94DB13FF91EF914398EF93FF938F
:10021000E6E4F0E00E94DB13FF91EF913A9531F7AD
:100220009923E1F680E0809311013A9A3B9A439832
:10023000A1E1B1E0119698E08E91983018F4392F31
:10024000992702C038E09850881F429808F4429AD3
:1002500000000000439AEF93FF93E6E4F0E00E9471
:10026000DB13FF91EF914398EF93FF93E6E4F0E007
:100270000E94DB13FF91EF913A9531F79923E1F654
:1002800080E2809311013A9A3B9A4398A1E1B1E050
:10029000119698E08E91983018F4392F992702C062
:1002A00038E09850881F429808F4429A00000000F5
:1002B000439AEF93FF93E6E4F0E00E94DB13FF9193
:1002C000EF914398EF93FF93E6E4F0E00E94DB1395
:1002D000FF91EF913A9531F79923E1F6419A4198D0
:1002E00070917A00706870937A005C9A01E010E077
:1002F00020E030E0AEE1B1E00D931D932D933C93EF
:1003000082E080931B010E944D0600917C00007EDC
:10031000066000937C000E942014AFEDB4E08D9342
:100320009C93AFEDB4E00D911C91003951E015079D
:1003300018F011F00C949E010C94A3015C98159890
:10034000479A0C94A7015C9A159A4798469A0E947E
:100350001116A8E7B1E035E00E94A5130E940E1621
:10036000A8E7B1E00E94D915AEE9B1E00D931C9366
:10037000AEE9B1E00D911C91023050E0150711F08B
:100380000C94C6010E94250C0C941D02003050E014
:10039000150711F00C94D0010E9454020C941D0218
:1003A000013050E0150711F00C94DA010E9454025C
:1003B0000C941D02033050E0150711F00C94E40179
:1003C0000E9454020C941D02043050E0150711F0F5
:1003D0000C94EE010E9454020C941D02083050E06F
:1003E000150711F00C94070200917C00007E076055
:1003F00000937C000E942014AFEDB4E08D939C9399
:1004000032E0AFEDB4E00E94C6130C941D02093037
:1004100050E0150711F00C941502E0EBFCE20E948D
:10042000BF130E94CB130C941D02033650E0150736
:1004300011F00C941D020C94007C0C9485010AE0D0
:1004400010E020E030E0AEE1B1E04D915D916D91C2
:100450007C910E94FD13A4EDB4E00D931D932D93A8
:100460003D9301E010E020E030E0A0EDB4E00D931A
:100470001D932D933C93A4EDB4E04D915D916D914E
:100480007C91A0EDB4E00D911D912D913C910E94C5
:10049000C6151CF011F00C945302A0EDB4E00E94BC
:1004A00074130C943B0208950E941116AEE7B1E05C
:1004B0003FE00E94A5130E940E160E941116ACE6A2
:1004C000B1E035E00E94A5130E940E160E9411169D
:1004D000A2E7B1E035E00E94A5130E940E160E942B
:1004E0001116AEE8B1E03FE00E94A5130E940E167F
:1004F000449A81E090E00E94E41344983A9A3B9A2F
:100500004398A0E0B1E0119698E08E91983018F4ED
:10051000392F992702C038E09850881F429808F474
:10052000429A00000000439AEF93FF93EFE0F0E05F
:100530000E94DB13FF91EF914398EF93FF93EFE05D
:10054000F0E00E94DB13FF91EF913A9531F7992388
:10055000E1F683ED809311013A9A3B9A4398A1E129
:10056000B1E0119698E08E91983018F4392F9927C0
:1005700002C038E09850881F429808F4429A000060
:100580000000439AEF93FF93E6E4F0E00E94DB1350
:10059000FF91EF914398EF93FF93E6E4F0E00E9420
:1005A000DB13FF91EF913A9531F79923E1F680E063
:1005B000809311013A9A3B9A4398A1E1B1E01196D8
:1005C00098E08E91983018F4392F992702C038E0BE
:1005D0009850881F429808F4429A00000000439AFD
:1005E000EF93FF93E6E4F0E00E94DB13FF91EF91BD
:1005F0004398EF93FF93E6E4F0E00E94DB13FF9152
:10060000EF913A9531F79923E1F680E0809311015B
:100610003A9A3B9A4398A1E1B1E0119698E08E9105
:10062000983018F4392F992702C038E09850881F65
:10063000429808F4429A00000000439AEF93FF9317
:10064000E6E4F0E00E94DB13FF91EF914398EF9313
:10065000FF93E6E4F0E00E94DB13FF91EF913A95FF
:1006600031F79923E1F6419A41983A9A3B9A439897
:10067000A2E0B1E0119698E08E91983018F4392FED
:10068000992702C038E09850881F429808F4429A8F
:1006900000000000439AEF93FF93E6E4F0E00E942D
:1006A000DB13FF91EF914398EF93FF93E6E4F0E0C3
:1006B0000E94DB13FF91EF913A9531F79923E1F610
:1006C00080E480930C013A9A3B9A4398ACE0B1E005
:1006D000119698E08E91983018F4392F992702C01E
:1006E00038E09850881F429808F4429A00000000B1
:1006F000439AEF93FF93E6E4F0E00E94DB13FF914F
:10070000EF914398EF93FF93E6E4F0E00E94DB1350
:10071000FF91EF913A9531F79923E1F63A9A3B9A96
:100720004398A4E1B1E0119698E08E91983018F4C6
:10073000392F992702C038E09850881F429808F452
:10074000429A00000000439AEF93FF93E6E4F0E042
:100750000E94DB13FF91EF914398EF93FF93E6E440
:10076000F0E00E94DB13FF91EF913A9531F7992366
:10077000E1F680E0809315013A9A3B9A4398A5E10F
:10078000B1E0119698E08E91983018F4392F99279E
:1007900002C038E09850881F429808F4429A00003E
:1007A0000000439AEF93FF93E6E4F0E00E94DB132E
:1007B000FF91EF914398EF93FF93E6E4F0E00E94FE
:1007C000DB13FF91EF913A9531F79923E1F682E03F
:1007D000809315013A9A3B9A4398A5E1B1E01196AE
:1007E00098E08E91983018F4392F992702C038E09C
:1007F0009850881F429808F4429A00000000439ADB
:10080000EF93FF93E6E4F0E00E94DB13FF91EF919A
:100810004398EF93FF93E6E4F0E00E94DB13FF912F
:10082000EF913A9531F79923E1F680E08093150135
:100830003A9A3B9A4398A5E1B1E0119698E08E91DF
:10084000983018F4392F992702C038E09850881F43
:10085000429808F4429A00000000439AEF93FF93F5
:10086000E6E4F0E00E94DB13FF91EF914398EF93F1
:10087000FF93E6E4F0E00E94DB13FF91EF913A95DD
:1008800031F79923E1F63A9A3B9A4398A2E0B1E016
:10089000119698E08E91983018F4392F992702C05C
:1008A00038E09850881F429808F4429A00000000EF
:1008B000439AEF93FF93E6E4F0E00E94DB13FF918D
:1008C000EF914398EF93FF93E6E4F0E00E94DB138F
:1008D000FF91EF913A9531F79923E1F680E8809303
:1008E0000C013A9A3B9A4398ACE0B1E0119698E03B
:1008F0008E91983018F4392F992702C038E098501B
:10090000881F429808F4429A00000000439AEF932F
:10091000FF93E6E4F0E00E94DB13FF91EF91439830
:10092000EF93FF93E6E4F0E00E94DB13FF91EF9179
:100930003A9531F79923E1F63A9A3B9A4398A4E124
:10094000B1E0119698E08E91983018F4392F9927DC
:1009500002C038E09850881F429808F4429A00007C
:100960000000439AEF93FF93E6E4F0E00E94DB136C
:10097000FF91EF914398EF93FF93E6E4F0E00E943C
:10098000DB13FF91EF913A9531F79923E1F680E07F
:10099000809315013A9A3B9A4398A5E1B1E01196EC
:1009A00098E08E91983018F4392F992702C038E0DA
:1009B0009850881F429808F4429A00000000439A19
:1009C000EF93FF93E6E4F0E00E94DB13FF91EF91D9
:1009D0004398EF93FF93E6E4F0E00E94DB13FF916E
:1009E000EF913A9531F79923E1F6AEE9B1E00D9137
:1009F0001C91003050E0150781E009F080E08F93F2
:100A0000AEE9B1E00D911C91033050E0150781E093
:100A100009F080E09F91892B8F93AEE9B1E00D91B1
:100A20001C91043050E0150781E009F080E09F91AF
:100A3000892B882311F40C94220581E08093150101
:100A40000C94250582E0809315013A9A3B9A4398CD
:100A5000A5E1B1E0119698E08E91983018F4392F05
:100A6000992702C038E09850881F429808F4429AAB
:100A700000000000439AEF93FF93E6E4F0E00E9449
:100A8000DB13FF91EF914398EF93FF93E6E4F0E0DF
:100A90000E94DB13FF91EF913A9531F79923E1F62C
:100AA00080E0809315013A9A3B9A4398A5E1B1E022
:100AB000119698E08E91983018F4392F992702C03A
:100AC00038E09850881F429808F4429A00000000CD
:100AD000439AEF93FF93E6E4F0E00E94DB13FF916B
:100AE000EF914398EF93FF93E6E4F0E00E94DB136D
:100AF000FF91EF913A9531F79923E1F6419A4198A8
:100B0000AEE7B1E00E94D915A4EAB1E00D931D93C0
:100B10002D933D93ACE6B1E00E94D915ADE0B1E074
:100B20000D931C93A2E7B1E00E94D915A0EAB1E0B1
:100B30000D931D932D933D93AEE8B1E00E94D9151E
:100B4000A8EAB1E00D931D932D933D93ACEDB4E075
:100B50000E94D915AFEDB4E00D931C93AEE9B1E05E
:100B60000D911C91003050E0150781E009F080E004
:100B70008F93AEE9B1E00D911C91033050E0150761
:100B800081E009F080E09F91892B8F93AEE9B1E07D
:100B90000D911C91043050E0150781E009F080E0D0
:100BA0009F91892B882311F40C94DA055D9828987D
:100BB0005B9A2998AEE9B1E00D911C91013050E0AB
:100BC000150711F00C94E8055D9A28985B98299810
:100BD000ECEAFCE20E94A215E0EAF1E00E94801437
:100BE0000E94A4140E94F114EDE0F0E0A6E1B1E04F
:100BF0000E940816E6E1F1E00E941716EDE0F0E031
:100C00000E944214AAE1B1E0DC9281E08093E10409
:100C100081E08093E10440911A010091E1040417FE
:100C200018F011F00C94210684E680931B010E94B9
:100C30004D06A1EEB4E08C918F5F8C9310F40C9470
:100C40000B06AAE1B1E00D91112744E650E00E94A5
:100C5000F313ACE1B1E00D931C93A0EAB1E00D9168
:100C60001C91ACE1B1E04D915C91041B150BACE122
:100C7000B1E00D931C93ACE1B1E00D911C910130FA
:100C800050E0150710F40C944B0680911C018093E2
:100C90001B010E944D06449A08954498159885E0DA
:100CA00090E00E94E41301E010E020E030E0ACEAC4
:100CB000B1E00D931D932D933C93ABE1B1E04C91CA
:100CC000552766277727ACEAB1E00D911D912D914C
:100CD0003C910E94C6151CF011F00C94CB0B3A9A73
:100CE0003B9A4398A2E0B1E0119698E08E9198303B
:100CF00018F4392F992702C038E09850881F42987D
:100D000008F4429A00000000439A00000000439853
:100D1000000000003A9591F7992341F780EC809309
:100D20000C013A9A3B9A4398ACE0B1E0119698E0F6
:100D30008E91983018F4392F992702C038E09850D6
:100D4000881F429808F4429A00000000439A00006D
:100D500000004398000000003A9591F7992341F76D
:100D60003A9A3B9A4398A1E0B1E0119698E08E91AF
:100D7000983018F4392F992702C038E09850881F0E
:100D8000429808F4429A00000000439A00000000D4
:100D90004398000000003A9591F7992341F73A9A59
:100DA0003B9A4398A4EAB1E0149690E28E91983071
:100DB00018F4392F992702C038E09850881F4298BC
:100DC00008F4429A00000000439A00000000439893
:100DD000000000003A9591F7992341F73A9A3B9A1F
:100DE0004398A3E0B1E0119698E08E91983018F402
:100DF000392F992702C038E09850881F429808F48C
:100E0000429A00000000439A00000000439800004E
:100E100000003A9591F7992341F780E090E0ADE02A
:100E2000B1E08D939C933A9A3B9A4398ADE0B1E040
:100E3000129690E18E91983018F4392F992702C0BC
:100E400038E09850881F429808F4429A0000000049
:100E5000439A000000004398000000003A9591F783
:100E6000992341F7419A41980E941F02AEE9B1E0EF
:100E70000D911C91013050E0150711F00C94A00762
:100E80002A982A9A2A9884EB94EFA2E1B1E08D93F4
:100E90009C9380E090E0ACEAB1E0AD90BD90AEEA0A
:100EA000B1E0AA0CBB1CAA0DBB1D8D939C93569A56
:100EB000579A5F98A2E1B1E012969EE08E91983029
:100EC00018F4392F992702C038E09850881F5E988F
:100ED00008F45E9A000000005F9A000000005F982E
:100EE000000000003A9591F7992341F72A9A2A9831
:100EF000579A52985F9A90E1ACEAB1E0AD90BD90FC
:100F0000AEEAB1E0AA0CBB1CAA0DBB1D129698302C
:100F100018F4392F992702C038E098505F980000E4
:100F2000000088944A990894881F5F9A0000000086
:100F30003A95A1F78E93992351F72A9A0C94EE07CC
:100F40002A9884EB90EFA2E1B1E08D939C93569A9E
:100F5000579A5F98A2E1B1E012969EE08E91983088
:100F600018F4392F992702C038E09850881F5E98EE
:100F700008F45E9A000000005F9A000000005F988D
:100F8000000000003A9591F7992341F72A9A2A9890
:100F9000579A52985F9A90E1ACEAB1E0AD90BD905B
:100FA000AEEAB1E0AA0CBB1CAA0DBB1D129698308C
:100FB00018F4392F992702C038E098505F98000044
:100FC000000088944A990894881F5F9A00000000E6
:100FD0003A95A1F78E93992351F72A9A3A9A3B9A18
:100FE0004398A2E0B1E0119698E08E91983018F401
:100FF000392F992702C038E09850881F429808F48A
:10100000429A00000000439A00000000439800004C
:1010100000003A9591F7992341F780E480930C0101
:101020003A9A3B9A4398ACE0B1E0119698E08E91E1
:10103000983018F4392F992702C038E09850881F4B
:10104000429808F4429A00000000439A0000000011
:101050004398000000003A9591F7992341F73A9A96
:101060003B9A4398A3E0B1E0119698E08E919830B6
:1010700018F4392F992702C038E09850881F4298F9
:1010800008F4429A00000000439A000000004398D0
:10109000000000003A9591F7992341F780E090E134
:1010A000ADE0B1E08D939C933A9A3B9A4398ADE0C2
:1010B000B1E0129690E18E91983018F4392F99276B
:1010C00002C038E09850881F429808F4429A000005
:1010D0000000439A000000004398000000003A9589
:1010E00091F7992341F7419A41980E941F02AEE976
:1010F000B1E00D911C91013050E0150711F00C94F6
:10110000E10884EB94EFA2E1B1E08D939C9380E041
:1011100090E0ACEAB1E0AD90BD90A6E7B2E0AA0CD9
:10112000BB1CAA0DBB1D8D939C932A982A9A2A98C2
:10113000569A579A5F98A2E1B1E012969EE08E917E
:10114000983018F4392F992702C038E09850881F3A
:101150005E9808F45E9A000000005F9A00000000AC
:101160005F98000000003A9591F7992341F72A9A79
:101170002A98579A52985F9A90E1ACEAB1E0AD9004
:10118000BD90A6E7B2E0AA0CBB1CAA0DBB1D12962F
:10119000983018F4392F992702C038E098505F989A
:1011A0000000000088944A990894881F5F9A000004
:1011B00000003A95A1F78E93992351F72A9A0C943F
:1011C0002F092A9884EB90EFA2E1B1E08D939C93D4
:1011D000569A579A5F98A2E1B1E012969EE08E91DE
:1011E000983018F4392F992702C038E09850881F9A
:1011F0005E9808F45E9A000000005F9A000000000C
:101200005F98000000003A9591F7992341F72A9AD8
:101210002A98579A52985F9A90E1ACEAB1E0AD9063
:10122000BD90A6E7B2E0AA0CBB1CAA0DBB1D12968E
:10123000983018F4392F992702C038E098505F98F9
:101240000000000088944A990894881F5F9A000063
:1012500000003A95A1F78E93992351F72A9A3A9A6A
:101260003B9A4398A2E0B1E0119698E08E919830B5
:1012700018F4392F992702C038E09850881F4298F7
:1012800008F4429A00000000439A000000004398CE
:10129000000000003A9591F7992341F780E480938C
:1012A0000C013A9A3B9A4398ACE0B1E0119698E071
:1012B0008E91983018F4392F992702C038E0985051
:1012C000881F429808F4429A00000000439A0000E8
:1012D00000004398000000003A9591F7992341F7E8
:1012E0003A9A3B9A4398A3E0B1E0119698E08E9128
:1012F000983018F4392F992702C038E09850881F89
:10130000429808F4429A00000000439A000000004E
:101310004398000000003A9591F7992341F780E047
:1013200090E2ADE0B1E08D939C933A9A3B9A43985A
:10133000ADE0B1E0129690E18E91983018F4392F1B
:10134000992702C038E09850881F429808F4429AC2
:1013500000000000439A00000000439800000000D5
:101360003A9591F7992341F7419A41980E941F02BB
:10137000AEE9B1E00D911C91013050E0150711F07C
:101380000C94220A84EB94EFA2E1B1E08D939C933C
:1013900080E090E0ACEAB1E0AD90BD90AEE3B3E0A8
:1013A000AA0CBB1CAA0DBB1D8D939C932A982A9A4C
:1013B0002A98569A579A5F98A2E1B1E012969EE059
:1013C0008E91983018F4392F992702C038E0985040
:1013D000881F5E9808F45E9A000000005F9A000083
:1013E00000005F98000000003A9591F7992341F7BB
:1013F0002A9A2A98579A52985F9A90E1ACEAB1E0FB
:10140000AD90BD90AEE3B3E0AA0CBB1CAA0DBB1D12
:101410001296983018F4392F992702C038E0985066
:101420005F980000000088944A990894881F5F9A8A
:10143000000000003A95A1F78E93992351F72A9A5C
:101440000C94700A2A9884EB90EFA2E1B1E08D939E
:101450009C93569A579A5F98A2E1B1E012969EE04B
:101460008E91983018F4392F992702C038E098509F
:10147000881F5E9808F45E9A000000005F9A0000E2
:1014800000005F98000000003A9591F7992341F71A
:101490002A9A2A98579A52985F9A90E1ACEAB1E05A
:1014A000AD90BD90AEE3B3E0AA0CBB1CAA0DBB1D72
:1014B0001296983018F4392F992702C038E09850C6
:1014C0005F980000000088944A990894881F5F9AEA
:1014D000000000003A95A1F78E93992351F72A9ABC
:1014E0003A9A3B9A4398A2E0B1E0119698E08E9127
:1014F000983018F4392F992702C038E09850881F87
:10150000429808F4429A00000000439A000000004C
:101510004398000000003A9591F7992341F780E441
:1015200080930C013A9A3B9A4398ACE0B1E0119653
:1015300098E08E91983018F4392F992702C038E03E
:101540009850881F429808F4429A00000000439A7D
:10155000000000004398000000003A9591F799239D
:1015600041F73A9A3B9A4398A3E0B1E0119698E08C
:101570008E91983018F4392F992702C038E098508E
:10158000881F429808F4429A00000000439A000025
:1015900000004398000000003A9591F7992341F725
:1015A00080E090E3ADE0B1E08D939C933A9A3B9A52
:1015B0004398ADE0B1E0129690E18E91983018F426
:1015C000392F992702C038E09850881F429808F4B4
:1015D000429A00000000439A000000004398000077
:1015E00000003A9591F7992341F7419A41980E945A
:1015F0001F02AEE9B1E00D911C91013050E01507DA
:1016000011F00C94630B84EB94EFA2E1B1E08D93A5
:101610009C9380E090E0ACEAB1E0AD90BD90A6E094
:10162000B4E0AA0CBB1CAA0DBB1D8D939C932A98F9
:101630002A9A2A98569A579A5F98A2E1B1E0129690
:101640009EE08E91983018F4392F992702C038E027
:101650009850881F5E9808F45E9A000000005F9A18
:10166000000000005F98000000003A9591F7992370
:1016700041F72A9A2A98579A52985F9A90E1ACEAD1
:10168000B1E0AD90BD90A6E0B4E0AA0CBB1CAA0DE1
:10169000BB1D1296983018F4392F992702C038E0F4
:1016A00098505F980000000088944A990894881F19
:1016B0005F9A000000003A95A1F78E93992351F7A5
:1016C0002A9A0C94B10B2A9884EB90EFA2E1B1E036
:1016D0008D939C93569A579A5F98A2E1B1E0129627
:1016E0009EE08E91983018F4392F992702C038E087
:1016F0009850881F5E9808F45E9A000000005F9A78
:10170000000000005F98000000003A9591F79923CF
:1017100041F72A9A2A98579A52985F9A90E1ACEA30
:10172000B1E0AD90BD90A6E0B4E0AA0CBB1CAA0D40
:10173000BB1D1296983018F4392F992702C038E053
:1017400098505F980000000088944A990894881F78
:101750005F9A000000003A95A1F78E93992351F704
:101760002A9AA4EAB1E00D911D912D913C91A8EA2D
:10177000B1E04D915D916D917C910E94C115A4EAFB
:10178000B1E00D931D932D933D93ACEAB1E00E941F
:1017900074130C945D06159A81E090E00E94E413A6
:1017A00000911B01003018F011F00C94D90B0C942F
:1017B000240C81E08093E20481E08093E204409174
:1017C0001B010091E204041718F011F00C94240C92
:1017D00032E0A2EEB4E0AD90BB24AEEAB1E0AA0CD8
:1017E000BB1CAA0DBB1D0E94C61332E0A2EEB4E0E2
:1017F000AD90BB24A6E7B2E0AA0CBB1CAA0DBB1D92
:101800000E94C61332E0A2EEB4E0AD90BB24AEE37A
:10181000B3E0AA0CBB1CAA0DBB1D0E94C61332E08C
:10182000A2EEB4E0AD90BB24A6E0B4E0AA0CBB1CD1
:10183000AA0DBB1D0E94C613A2EEB4E08C918F5F6F
:101840008C9310F40C94DF0B089544980E941116A9
:10185000A2E2B1E03FE00E94A5130E940E160E9492
:101860001116A2E3B1E03FE00E94A5130E940E16FC
:101870000E941116A2E4B1E036E00E94A5130E9476
:101880000E160E941116A9E4B1E035E00E94A513DE
:101890000E940E160E941116AFE4B1E036E00E94DD
:1018A000A5130E940E160E941116A6E5B1E036E0BF
:1018B0000E94A5130E940E16A2E2B1E00E94D91563
:1018C000ADE5B1E00D931D932D933D93A2E3B1E0FF
:1018D0000E94D915A1E6B1E00D931D932D933D9380
:1018E000A2E4B1E00E94D915A5E6B1E00D931C93E6
:1018F000A9E4B1E00E94D915A7E6B1E00C93AFE4EA
:10190000B1E00E94D915A8E6B1E00D931C93A6E5BD
:10191000B1E00E94D915AAE6B1E00D931C935D9841
:10192000289A5B9A299A8AE090E00E94E413449AEC
:101930008AE090E00E94E41344988AE090E00E94DC
:10194000E4133A9A3B9A4398A0E0B1E0119698E0EC
:101950008E91983018F4392F992702C038E09850AA
:10196000881F429808F4429A00000000439AEF93BF
:10197000FF93EFE0F0E00E94DB13FF91EF914398BB
:10198000EF93FF93EFE0F0E00E94DB13FF91EF9104
:101990003A9531F79923E1F683ED809311013A9A54
:1019A0003B9A4398A1E1B1E0119698E08E9198306E
:1019B00018F4392F992702C038E09850881F4298B0
:1019C00008F4429A00000000439AEF93FF93E6E484
:1019D000F0E00E94DB13FF91EF914398EF93FF93A8
:1019E000E6E4F0E00E94DB13FF91EF913A9531F7C6
:1019F0009923E1F680E0809311013A9A3B9A43984B
:101A0000A1E1B1E0119698E08E91983018F4392F49
:101A1000992702C038E09850881F429808F4429AEB
:101A200000000000439AEF93FF93E6E4F0E00E9489
:101A3000DB13FF91EF914398EF93FF93E6E4F0E01F
:101A40000E94DB13FF91EF913A9531F79923E1F66C
:101A500080E2809311013A9A3B9A4398A1E1B1E068
:101A6000119698E08E91983018F4392F992702C07A
:101A700038E09850881F429808F4429A000000000D
:101A8000439AEF93FF93E6E4F0E00E94DB13FF91AB
:101A9000EF914398EF93FF93E6E4F0E00E94DB13AD
:101AA000FF91EF913A9531F79923E1F6419A4198E8
:101AB0003A9A3B9A4398A2E0B1E0119698E08E9151
:101AC000983018F4392F992702C038E09850881FB1
:101AD000429808F4429A00000000439AEF93FF9363
:101AE000E6E4F0E00E94DB13FF91EF914398EF935F
:101AF000FF93E6E4F0E00E94DB13FF91EF913A954B
:101B000031F79923E1F680EC80930C013A9A3B9AE5
:101B10004398ACE0B1E0119698E08E91983018F4BB
:101B2000392F992702C038E09850881F429808F44E
:101B3000429A00000000439AEF93FF93E6E4F0E03E
:101B40000E94DB13FF91EF914398EF93FF93E6E43C
:101B5000F0E00E94DB13FF91EF913A9531F7992362
:101B6000E1F63A9A3B9A4398A4E1B1E0119698E0E5
:101B70008E91983018F4392F992702C038E0985088
:101B8000881F429808F4429A00000000439AEF939D
:101B9000FF93E6E4F0E00E94DB13FF91EF9143989E
:101BA000EF93FF93E6E4F0E00E94DB13FF91EF91E7
:101BB0003A9531F79923E1F680E0809315013A9A3E
:101BC0003B9A4398A5E1B1E0119698E08E91983048
:101BD00018F4392F992702C038E09850881F42988E
:101BE00008F4429A00000000439AEF93FF93E6E462
:101BF000F0E00E94DB13FF91EF914398EF93FF9386
:101C0000E6E4F0E00E94DB13FF91EF913A9531F7A3
:101C10009923E1F680916701809315013A9A3B9AE6
:101C20004398A5E1B1E0119698E08E91983018F4B0
:101C3000392F992702C038E09850881F429808F43D
:101C4000429A00000000439AEF93FF93E6E4F0E02D
:101C50000E94DB13FF91EF914398EF93FF93E6E42B
:101C6000F0E00E94DB13FF91EF913A9531F7992351
:101C7000E1F680E2809315013A9A3B9A4398A5E1F8
:101C8000B1E0119698E08E91983018F4392F992789
:101C900002C038E09850881F429808F4429A000029
:101CA0000000439AEF93FF93E6E4F0E00E94DB1319
:101CB000FF91EF914398EF93FF93E6E4F0E00E94E9
:101CC000DB13FF91EF913A9531F79923E1F6419AB1
:101CD00081E090E00E94E4134198A1E6B1E04D91CB
:101CE0005D916D917C91ADE5B1E00D911D912D91CE
:101CF0003C910E94C61511F00C94290F3A9A3B9A18
:101D00004398A2E0B1E0119698E08E91983018F4D3
:101D1000392F992702C038E09850881F429808F45C
:101D2000429A00000000439A00000000439800001F
:101D300000003A9591F7992341F780EC80930C01CC
:101D40003A9A3B9A4398ACE0B1E0119698E08E91B4
:101D5000983018F4392F992702C038E09850881F1E
:101D6000429808F4429A00000000439AEF93FF93D0
:101D7000E6E4F0E00E94DB13FF91EF914398EF93CC
:101D8000FF93E6E4F0E00E94DB13FF91EF913A95B8
:101D900031F79923E1F63A9A3B9A4398A1E0B1E0F2
:101DA000119698E08E91983018F4392F992702C037
:101DB00038E09850881F429808F4429A00000000CA
:101DC000439AEF93FF93E6E4F0E00E94DB13FF9168
:101DD000EF914398EF93FF93E6E4F0E00E94DB136A
:101DE000FF91EF913A9531F79923E1F63A9A3B9AB0
:101DF0004398ADE5B1E0149690E28E91983018F4D6
:101E0000392F992702C038E09850881F429808F46B
:101E1000429A00000000439AEF93FF93E6E4F0E05B
:101E20000E94DB13FF91EF914398EF93FF93E6E459
:101E3000F0E00E94DB13FF91EF913A9531F799237F
:101E4000E1F6419A81E090E00E94E41341980C94FD
:101E50007B103A9A3B9A4398A2E0B1E0119698E041
:101E60008E91983018F4392F992702C038E0985095
:101E7000881F429808F4429A00000000439A00002C
:101E800000004398000000003A9591F7992341F72C
:101E900080E880930C013A9A3B9A4398ACE0B1E019
:101EA000119698E08E91983018F4392F992702C036
:101EB00038E09850881F429808F4429A00000000C9
:101EC000439AEF93FF93E6E4F0E00E94DB13FF9167
:101ED000EF914398EF93FF93E6E4F0E00E94DB1369
:101EE000FF91EF913A9531F79923E1F63A9A3B9AAF
:101EF0004398A1E0B1E0119698E08E91983018F4E3
:101F0000392F992702C038E09850881F429808F46A
:101F1000429A00000000439AEF93FF93E6E4F0E05A
:101F20000E94DB13FF91EF914398EF93FF93E6E458
:101F3000F0E00E94DB13FF91EF913A9531F799237E
:101F4000E1F63A9A3B9A4398ADE5B1E0149690E2F7
:101F50008E91983018F4392F992702C038E09850A4
:101F6000881F429808F4429A00000000439AEF93B9
:101F7000FF93E6E4F0E00E94DB13FF91EF914398BA
:101F8000EF93FF93E6E4F0E00E94DB13FF91EF9103
:101F90003A9531F79923E1F6419A81E090E00E9469
:101FA000E41341983A9A3B9A4398A2E0B1E0119623
:101FB00098E08E91983018F4392F992702C038E0B4
:101FC0009850881F429808F4429A00000000439AF3
:101FD000000000004398000000003A9591F7992313
:101FE00041F780E480930C013A9A3B9A4398ACE025
:101FF000B1E0119698E08E91983018F4392F992716
:1020000002C038E09850881F429808F4429A0000B5
:102010000000439AEF93FF93E6E4F0E00E94DB13A5
:10202000FF91EF914398EF93FF93E6E4F0E00E9475
:10203000DB13FF91EF913A9531F79923E1F63A9A44
:102040003B9A4398A1E0B1E0119698E08E919830C8
:1020500018F4392F992702C038E09850881F429809
:1020600008F4429A00000000439AEF93FF93E6E4DD
:10207000F0E00E94DB13FF91EF914398EF93FF9301
:10208000E6E4F0E00E94DB13FF91EF913A9531F71F
:102090009923E1F63A9A3B9A4398A1E6B1E0149667
:1020A00090E28E91983018F4392F992702C038E0C9
:1020B0009850881F429808F4429A00000000439A02
:1020C000EF93FF93E6E4F0E00E94DB13FF91EF91C2
:1020D0004398EF93FF93E6E4F0E00E94DB13FF9157
:1020E000EF913A9531F79923E1F6419A81E090E03A
:1020F0000E94E41341983A9A3B9A4398A2E0B1E0D7
:10210000119698E08E91983018F4392F992702C0D3
:1021100038E09850881F429808F4429A0000000066
:10212000439AEF93FF93E6E4F0E00E94DB13FF9104
:10213000EF914398EF93FF93E6E4F0E00E94DB1306
:10214000FF91EF913A9531F79923E1F680E480937E
:102150000C013A9A3B9A4398ACE0B1E0119698E0B2
:102160008E91983018F4392F992702C038E0985092
:10217000881F429808F4429A00000000439AEF93A7
:10218000FF93E6E4F0E00E94DB13FF91EF914398A8
:10219000EF93FF93E6E4F0E00E94DB13FF91EF91F1
:1021A0003A9531F79923E1F63A9A3B9A4398A3E09E
:1021B000B1E0119698E08E91983018F4392F992754
:1021C00002C038E09850881F429808F4429A0000F4
:1021D0000000439AEF93FF93E6E4F0E00E94DB13E4
:1021E000FF91EF914398EF93FF93E6E4F0E00E94B4
:1021F000DB13FF91EF913A9531F79923E1F63A9A83
:102200003B9A4398A5E6B1E0129690E18E91983002
:1022100018F4392F992702C038E09850881F429847
:1022200008F4429A00000000439AEF93FF93E6E41B
:10223000F0E00E94DB13FF91EF914398EF93FF933F
:10224000E6E4F0E00E94DB13FF91EF913A9531F75D
:102250009923E1F6419A81E090E00E94E4134198CD
:10226000809168018093E40486E08093E504809186
:1022700068018093E4043A9A3B9A4398A2E0B1E063
:10228000119698E08E91983018F4392F992702C052
:1022900038E09850881F429808F4429A00000000E5
:1022A000439AEF93FF93E6E4F0E00E94DB13FF9183
:1022B000EF914398EF93FF93E6E4F0E00E94DB1385
:1022C000FF91EF913A9531F79923E1F680E48093FD
:1022D0000C013A9A3B9A4398ACE0B1E0119698E031
:1022E0008E91983018F4392F992702C038E0985011
:1022F000881F429808F4429A00000000439AEF9326
:10230000FF93E6E4F0E00E94DB13FF91EF91439826
:10231000EF93FF93E6E4F0E00E94DB13FF91EF916F
:102320003A9531F79923E1F63A9A3B9A4398A5EE0C
:10233000B4E0119698E08E91983018F4392F9927CF
:1023400002C038E09850881F429808F4429A000072
:102350000000439AEF93FF93E6E4F0E00E94DB1362
:10236000FF91EF914398EF93FF93E6E4F0E00E9432
:10237000DB13FF91EF913A9531F79923E1F680E075
:102380008093E3043A9A3B9A4398A3EEB4E0119603
:1023900098E08E91983018F4392F992702C038E0D0
:1023A0009850881F429808F4429A00000000439A0F
:1023B000EF93FF93E6E4F0E00E94DB13FF91EF91CF
:1023C0004398EF93FF93E6E4F0E00E94DB13FF9164
:1023D000EF913A9531F79923E1F698E0A8E6B1E05C
:1023E0000E9437140091680140E1040FA3EEB4E0AD
:1023F0000C933A9A3B9A4398A3EEB4E0119698E076
:102400008E91983018F4392F992702C038E09850EF
:10241000881F429808F4429A00000000439AEF9304
:10242000FF93E6E4F0E00E94DB13FF91EF91439805
:10243000EF93FF93E6E4F0E00E94DB13FF91EF914E
:102440003A9531F79923E1F63A9A3B9A4398A4EEEC
:10245000B4E0119698E08E91983018F4392F9927AE
:1024600002C038E09850881F429808F4429A000051
:102470000000439AEF93FF93E6E4F0E00E94DB1341
:10248000FF91EF914398EF93FF93E6E4F0E00E9411
:10249000DB13FF91EF913A9531F79923E1F6419AD9
:1024A00081E090E00E94E413419880916A0180935A
:1024B000E4043A9A3B9A4398A2E0B1E0119698E07E
:1024C0008E91983018F4392F992702C038E098502F
:1024D000881F429808F4429A00000000439AEF9344
:1024E000FF93E6E4F0E00E94DB13FF91EF91439845
:1024F000EF93FF93E6E4F0E00E94DB13FF91EF918E
:102500003A9531F79923E1F680E880930C013A9AE5
:102510003B9A4398ACE0B1E0119698E08E919830E8
:1025200018F4392F992702C038E09850881F429834
:1025300008F4429A00000000439AEF93FF93E6E408
:10254000F0E00E94DB13FF91EF914398EF93FF932C
:10255000E6E4F0E00E94DB13FF91EF913A9531F74A
:102560009923E1F63A9A3B9A4398A5EEB4E0119686
:1025700098E08E91983018F4392F992702C038E0EE
:102580009850881F429808F4429A00000000439A2D
:10259000EF93FF93E6E4F0E00E94DB13FF91EF91ED
:1025A0004398EF93FF93E6E4F0E00E94DB13FF9182
:1025B000EF913A9531F79923E1F680E08093E304B7
:1025C0003A9A3B9A4398A3EEB4E0119698E08E9124
:1025D000983018F4392F992702C038E09850881F96
:1025E000429808F4429A00000000439AEF93FF9348
:1025F000E6E4F0E00E94DB13FF91EF914398EF9344
:10260000FF93E6E4F0E00E94DB13FF91EF913A952F
:1026100031F79923E1F698E0AAE6B1E00E94371479
:1026200000916A0140E1040FA3EEB4E00C933A9AE2
:102630003B9A4398A3EEB4E0119698E08E919830BF
:1026400018F4392F992702C038E09850881F429813
:1026500008F4429A00000000439AEF93FF93E6E4E7
:10266000F0E00E94DB13FF91EF914398EF93FF930B
:10267000E6E4F0E00E94DB13FF91EF913A9531F729
:102680009923E1F63A9A3B9A4398A4EEB4E0119666
:1026900098E08E91983018F4392F992702C038E0CD
:1026A0009850881F429808F4429A00000000439A0C
:1026B000EF93FF93E6E4F0E00E94DB13FF91EF91CC
:1026C0004398EF93FF93E6E4F0E00E94DB13FF9161
:1026D000EF913A9531F79923E1F6419A81E090E044
:1026E0000E94E413419808950D911D912D913C9104
:1026F0000F5F1F4F2F4F3F4F3C932E931E930E9310
:10270000089505D00E94F31300FC0CD00895002416
:10271000E89457FF02C009D0689400F80BD010F875
:102720000124089502D009D00895509540954F5F37
:102730005F4F0895E89417FF0895009510950F5F77
:102740001F4F68940895A8EAB0E112D08D3039F097
:102750003323D9F38D933A9563FE20D0F6CF63FCF3
:1027600004C08DE01BD08AE019D088278C9308958F
:102770008091C00087FFFCCF8091C60008950E9421
:102780009E15802D11F00AD0FACF08958D9106D0B4
:102790003A95E1F708958DE001D08AE00090C000FD
:1027A00005FEFCCF8093C600089588EE93E00CD020
:1027B0003197D9F708953197F1F70895689462F841
:1027C0000895E89462F80895EF93FF93EE27E82BBD
:1027D000E92B31F0E6E6FEE03197F1F70197D1F70A
:1027E000FF91EF9108950F92B801469F8001479F96
:1027F000100D569F100D0F9008950F921F922F925B
:10280000C801D901489F80014A9F90014B9F202C0D
:10281000499F100D211D321D5A9F202C589F100DCD
:10282000211D321D599F200D311D689F200D311D26
:10283000699F300D789F300D2F901F900F90089555
:1028400070917A00706470937A0000907A0006FCB0
:10285000FCCF70917A00706470937A0000907A00D7
:1028600006FCFCCF8091780090917900089590301B
:1028700041F00D911C91169507959A95E1F71C93DF
:102880000E9308953DD0992711278F2D880F80E84A
:10289000F82A802F881F08F41FEF41F08F57082F68
:1028A00007FD04C0003240F08FEF01C08827982F49
:1028B000D82EE82EF82E09C08FE1801B082FF69441
:1028C000E794D79497950A95D1F7112351F09095F5
:1028D000D094E094F09481E0980F8827D81EE81EE9
:1028E000F81E0F2DFE2CED2CD92E0895D094E094D7
:1028F000F09491E0D90E9927E91EF91E10950895DC
:10290000D190E190F19001910895219131914191FF
:1029100051910895102F90E8FF0C001F0927990F7F
:10292000F7941078652F90E8440F551F5927990F99
:102930004795607800380895FF0C90E89027110FB4
:102940009795F794092F0895102FBD2CDE2CEF2CAE
:10295000F02E11234AF4B094D094E094F0949FEFB9
:10296000B91AD90AE90AF90A0EE1FF2039F4FE2C56
:10297000ED2CDB2CBB240850C2F767C032F00A955F
:10298000BB0CDD1CEE1CFF1CF9CF0E94C814D4CF79
:10299000B7FE089590E8B91611F4D0FE08959FEFA0
:1029A000D91AE90AF90A09F403950895502F2D2D33
:1029B0003E2D4F2D612F08952DEC3CEC4CEC5DE34A
:1029C00066270FC09DDFF2DFDD24EE2490E8F92EAC
:1029D0000FE307C09ADF05C02227332740E251E406
:1029E0006627552351F1002381F194DF71F11627F9
:1029F000005850580894050B18F407FD03C025C073
:102A000007FD23C0469537952795F694E794D7940C
:102A100022D0FF202AF0DD0CEE1CFF1C015073F0C9
:102A20009D2D969548F0DD203AF4EE202AF491E0B1
:102A3000D90E9927E91EF91E7FCF07C09FE7092FFE
:102A4000F92A9FEFD92EE92E0895DD24EE24FF24E4
:102A50000027112708959F929924AA24BB2488E176
:102A6000D216E306F40628F0D21AE30AF40A089410
:102A700001C08894991CAA1CBB1CDD0CEE1CFF1C19
:102A80008A9571F7D92CEA2CFB2C9F9008950AF0B7
:102A900045D052CF5FE322273327442701C035DFDB
:102AA00039DF5038B1F3003899F3902F951B8BF331
:102AB00012F434D0FACF983118F022273327442764
:102AC000983028F0232F342F44279850F9CF99239A
:102AD00029F04695379527959A95D9F7912F9627FE
:102AE00042F014D0B0F6F794E794D7940F5F8BF6CA
:102AF000A5CF10D051F008F4F9DEFF2052F2DD0C22
:102B0000EE1CFF1C0150CBF799CF9FCFD20EE31ED6
:102B1000F41E0895D21AE30AF40A0895DF92EF92A0
:102B2000FF920F931F93D22EE32EF42E052F162F14
:102B30006F915F914F913F912F910895C895319674
:102B400000200895FBDF202DF9DF302DF7DF402D29
:102B5000F5DF502D089507FB00680EF40F7757FB43
:102B600050680EF45F7707FD02C057FF05C0D2160C
:102B7000E306F406050708952D153E054F05500799
:102B80000895040F151F261F371F089504171507F2
:102B9000260737070895000F111F221F331F0895BE
:102BA00000951095209530950F5F1F4F2F4F3F4F89
:102BB000089500271127222733271DD08A3328F4B0
:102BC000803318F005D015D0F9CF0EF4E9CF089571
:102BD00080538F93402F512F622F732FDCDFDBDF69
:102BE000D0DFD9DF8F919927080F191F291F391FAF
:102BF00008958D910895E894FCDF8032E9F38B32DB
:102C0000D9F38930C9F38D3211F46894F2CF089565
:102C100094E081918D939A95E1F70895E89463F893
:102C20000895689463F808956BDE80E003C068DE61
:102C3000802F8078882321F0DF92EF92FF920F930C
:102C40008F9368DE802F839512F4FFDE1BC0809582
:102C50008A95885E0AF415C088501AF40CD0D922DF
:102C600010C0DD2488501AF406D0E9220AC0EE24F0
:102C700002D0F92206C09FEF8770990F8A95EAF774
:102C800008955ADE8F918823D9F35F914F913F9138
:102C90002F910F9360DF0F9199F390F302D050685A
:102CA000FFCE5FE340E83327222708950000C842A3
:102CB0004649524D574152452056312E353020302D
:0C2CC000322D30312D3230313320000035
:00000001FF
